:100000000C9446000C9463000C9463000C94630001
:100010000C9463000C9463000C9463000C946300D4
:100020000C9463000C9463000C9463000C946300C4
:100030000C9463000C9463000C9463000C948C008B
:100040000C9463000C9463000C9463000C946300A4
:100050000C9463000C949C000C9463000C9463005B
:100060000C9463000C9463000C9463000C94630084
:100070000C9463000C9463000C9463000C94630074
:100080000C9463000C9463000C94630011241FBE55
:10009000CFEFD0E1DEBFCDBF11E0A0E0B1E0E4E5FD
:1000A000F4E100E00BBF02C007900D92A830B10749
:1000B000D9F711E0A8E0B1E001C01D92AA31B10763
:1000C000E1F70C94DF000C940000CF93DF93CDB7E1
:1000D000DEB7F8948FEF80933A008FEF80933B0068
:1000E0008FEF809334008FEF809335008091500024
:1000F0008860809350008FE18093530082E080936A
:1001000051008091570082608093570078940E943C
:10011000E900DF91CF9108951F920F920FB60F92D1
:100120001124CF93DF93CDB7DEB7DF91CF910F903E
:100130000FBE0F901F9018951F920F920FB60F923F
:1001400011242F933F934F935F936F937F938F93DC
:100150009F93AF93BF93EF93FF93CF93DF93CDB76D
:10016000DEB70E945601DF91CF91FF91EF91BF91D1
:10017000AF919F918F917F916F915F914F913F913F
:100180002F910F900FBE0F901F901895CF93DF9374
:10019000CDB7DEB721970FB6F894DEBF0FBECDBF47
:1001A0000E946500809114018823E1F3809114017D
:1001B00089834FEF60E089810E949002F3CFCFEFF7
:1001C000D0E1DEBFCDBF0E94C60080E090E00C947D
:1001D000290ACF93DF93CDB7DEB78CEA8093260050
:1001E00080E68093270066E086E290E00E940102AC
:1001F00082E38093130110920C0180910C018430F2
:1002000078F480910C019927FC01E85FFE4F809102
:100210001301808380910C018F5F80930C01EDCFDF
:1002200080E180930D011092140110921201DF9170
:10023000CF910895CF93DF93CDB7DEB722970FB656
:10024000F894DEBF0FBECDBF89836A838981992769
:10025000FC01E25FFE4F8A81808322960FB6F894FC
:10026000DEBF0FBECDBFDF91CF910895CF93DF9357
:10027000CDB7DEB721970FB6F894DEBF0FBECDBF66
:1002800089839CEF80912700892380932700909198
:1002900027008981890F8093270021960FB6F89453
:1002A000DEBF0FBECDBFDF91CF910895CF93DF9317
:1002B000CDB7DEB723970FB6F894DEBF0FBECDBF24
:1002C000809125008093130180912700837089839A
:1002D0008981282F33273B832A838A819B81813020
:1002E0009105F9F0EA81FB81E230F10534F42A81CD
:1002F0003B812115310561F02EC08A819B818230BE
:100300009105C1F0EA81FB81E330F105E1F023C002
:100310006091130180E00E941A0181E00E94360181
:100320001AC06091130181E00E941A0182E00E94CC
:10033000360111C06091130182E00E941A0183E02E
:100340000E94360108C06091130183E00E941A01E7
:1003500080E00E94360119828981843038F58981D4
:100360009927DC01A25FBE4F89819927FC01E85FD4
:10037000FE4F9C9180818917A8F4898199279C015F
:100380002A5E3E4F89819927DC01A25FBE4F898199
:100390009927FC01E85FFE4F9C918081981B892F73
:1003A000F901808389818F5F8983D6CF10921401F0
:1003B00010921201198289818430D0F48091120147
:1003C0008F3FB1F089819927FC01EA5EFE4F908151
:1003D00080910D01891740F48FEF8093120169819C
:1003E00084E191E00E94010289818F5F8983E3CFDC
:1003F00023960FB6F894DEBF0FBECDBFDF91CF912D
:100400000895CF93DF93CDB7DEB724970FB6F89456
:10041000DEBF0FBECDBF9A8389836B838B81282F6C
:10042000332781E090E002C0880F991F2A95E2F7F8
:100430008C83A981BA81E981FA8190818C81892B91
:100440008C9324960FB6F894DEBF0FBECDBFDF911C
:10045000CF910895CF93DF93CDB7DEB725970FB631
:10046000F894DEBF0FBECDBF9A8389836B838B81E7
:10047000282F332781E090E0022E02C0880F991FB9
:100480000A94E2F78C838C81882321F48C8181701B
:100490008D8301C01D828D818C83A981BA81E98100
:1004A000FA8190818C81892B8C9325960FB6F894D4
:1004B000DEBF0FBECDBFDF91CF910895CF93DF9305
:1004C000CDB7DEB723970FB6F894DEBF0FBECDBF12
:1004D00089836A838A81282F332781E090E002C0D4
:1004E000880F991F2A95E2F78B8399818B81892345
:1004F00089838981282F33278A81992702C03595DE
:1005000027958A95E2F7C9018983898199272396DE
:100510000FB6F894DEBF0FBECDBFDF91CF91089527
:10052000CF93DF93CDB7DEB723970FB6F894DEBF36
:100530000FBECDBF89836A834B838B818F3F29F4A4
:100540008FEF9981891B80933B0023960FB6F89417
:10055000DEBF0FBECDBFDF91CF910895CF93DF9364
:10056000CDB7DEB760970FB6F894DEBF0FBECDBF34
:1005700069837A838B839C8320E030E040E452E4FB
:1005800069817A818B819C810E947906DC01CB0193
:10059000BC01CD010E94AA03DC01CB018D831E8228
:1005A0009E818D81981708F04AC089819A81AB811C
:1005B000BC818F839887A987BA872BEA3AEA4AEAEF
:1005C00050E46F81788589859A850E945E05DC01FB
:1005D000CB018C879D87AE87BF8720E030E040E865
:1005E0005FE36C857D858E859F850E9495078823B6
:1005F0000CF003C081E08B8718C020E030E04FE7AB
:1006000053E46C857D858E859F850E942907181689
:100610000CF002C01B8609C06C857D858E859F8588
:100620000E94AA03DC01CB018B878B85888B88898C
:100630008A95F1F7888B8E818F5F8E83B1CF60961C
:100640000FB6F894DEBF0FBECDBFDF91CF910895F6
:10065000CF93DF93CDB7DEB762970FB6F894DEBFC6
:100660000FBECDBF69837A838B839C8320E030E00B
:1006700040E851E469817A818B819C810E947906EE
:10068000DC01CB01BC01CD010E94AA03DC01CB013E
:100690008D831E829E818D81981708F052C08981BA
:1006A0009A81AB81BC818F839887A987BA8720E024
:1006B00030E04AE755E46F81788589859A850E9404
:1006C0005E05DC01CB018D879E87AF87B88B20E06C
:1006D00030E040E85FE36D857E858F8598890E94D4
:1006E000950788230CF005C081E090E09C878B87FC
:1006F0001AC020E03FEF4FE757E46D857E858F8578
:1007000098890E94290718160CF003C01C861B86C6
:100710000AC06D857E858F8598890E94AA03DC01B9
:10072000CB019C878B878B859C859A8B898B89894C
:100730009A890197F1F79A8B898B8E818F5F8E83CF
:10074000A9CF62960FB6F894DEBF0FBECDBFDF9182
:10075000CF910895EF92FF920F931F937B018C012D
:1007600020E030E040E05FE40E945F0788239CF0D7
:1007700020E030E040E05FECC801B7010E94F804DF
:10078000DC01CB01BC01CD010E94CB076050704061
:100790008040904804C0C801B7010E94CB071F9158
:1007A0000F91FF90EF900895A0E0B0E0EAEDF3E044
:1007B0000C94F2098C017B015A01DC018C9182308E
:1007C00058F0FB019081923010F4A7010BC18430E6
:1007D00029F4943009F4A6C0A80104C19430A9F307
:1007E000923009F4A9C0823081F3F801C280D3802D
:1007F000FB0162817381F801248135814681578133
:10080000F7016480758086809780C601861B970BF0
:1008100097FDD8C080970CF46CC06C157D050CF06A
:10082000ADC0662477244301F8016181F70181811D
:10083000681709F499C0662309F491C0621A730A13
:10084000840A950AA401930157FDC0C0F5011182E5
:10085000B60119012A0179018A0139014A01089476
:100860006108710881089108FFEF6F16FFEF7F069E
:10087000FFEF8F06FFE39F06F0F4A8019701220F18
:10088000331F441F551F19012A01B60161507040E2
:100890006B0179018A0139014A01089461087108E4
:1008A000810891088FEF68168FEF78068FEF880622
:1008B0008FE3980610F383E0D5018C9357FC64C056
:1008C000F501248335834683578373836283A501AF
:1008D00089C06F5F7F4FD401C30181709070A07099
:1008E000B0709694879477946794682A792A8A2AB4
:1008F0009B2A6C157D056CF311C00894C11CD11C9A
:10090000DA01C90181709070A070B070569547955A
:1009100037952795282B392B4A2B5B2BC616D706E4
:1009200064F382CFF8019181FB018181981709F46A
:1009300053CF40E051E056C0823009F04DCFDA018C
:10094000F80188E001900D928150E1F7F801818172
:10095000F70191818923F5018183A50143C02619FF
:1009600037094809590970CFF5016183B601260D91
:10097000371D481D591D19012A019DCF6B0120E02B
:1009800030E040E050E050CFD201C101B695A795CC
:100990009795879521E030E040E050E02222332215
:1009A00044225522282A392A4A2A5B2AF501248220
:1009B0003582468257820894C11CD11CD382C282E0
:1009C000A50110C0909581959F4F24CF81E0F5013E
:1009D0008183B60150954095309521953F4F4F4FFB
:1009E0005F4F37CFCA01E2E1CDB7DEB70C940E0AF4
:1009F000A0E2B0E0EEEFF4E00C94000ADC01CB01E1
:100A0000898F9A8FAB8FBC8F2D8F3E8F4F8F58A3BE
:100A1000BE016F5F7F4FCE0149960E9405098E018E
:100A2000075F1F4FB801CE014D960E940509AE0128
:100A30004F5E5F4FB801CE0101960E94D4030E9421
:100A40001D08DC01CB01BC01CD01E4E0A0960C94B3
:100A50001C0AA0E2B0E0EFE2F5E00C94000ADC0131
:100A6000CB01898F9A8FAB8FBC8F2D8F3E8F4F8F8D
:100A700058A3BE016F5F7F4FCE0149960E940509C2
:100A80008E01075F1F4FB801CE014D960E940509E8
:100A90008A8591E089278A87AE014F5E5F4FB80152
:100AA000CE0101960E94D4030E941D08DC01CB01F7
:100AB000BC01CD01E4E0A0960C941C0AA0E2B0E0D9
:100AC000E4E6F5E00C94F209DC01CB01898F9A8F02
:100AD000AB8FBC8F2D8F3E8F4F8F58A3BE016F5FA2
:100AE0007F4FCE0149960E94050969E070E06C0FC6
:100AF0007D1FCE014D960E940509FE0131966624A8
:100B000077244301130124018981823098F099856B
:100B1000923058F420E091818A85981321E02A8749
:100B200069E070E06C0F7D1FD9C0843059F49230B9
:100B300009F45BC020E091818A85981321E021832C
:100B4000BF01CCC0943009F44DC0823099F392308B
:100B500009F3ED80FE800F8118852D853E854F8538
:100B60005889640153016FE170E00CC0220F331FFC
:100B7000441F551F16950795F794E79461507040F0
:100B800077FD36C0D801C70181709070A070B07039
:100B9000892BC9F080E090E0220E331E441E551EC2
:100BA000221633064406550610F481E090E0AA2789
:100BB00097FDA095BA2F8A0D9B1DAC1DBD1D680E1B
:100BC000791E8A1E9B1EAA0CBB1CCC1CDD1C57FF69
:100BD000CDCF81E090E0A0E0B0E0A82AB92ACA2AEF
:100BE000DB2AC4CF823009F095CF60E071E076C097
:100BF000228133818B859C85280F391F2E5F3F4FC3
:100C0000A90160E091818A85981361E06A8B97FE63
:100C10000FC02FC0CA010197AC019C01660C771C64
:100C2000881C991C57FC41C0220C331C441C551CC9
:100C300090E0691690E0790690E0890690E49906C4
:100C400048F33C8B2B8BD401C3018F779070A0703D
:100C5000B07080349105A105B10581F16D8A7E8A5D
:100C60008F8A988E83E0898B61E170E06C0F7D1F25
:100C700035C02F5F3F4FA901D401C301817090702F
:100C8000A070B070892B61F05694479437942794E4
:100C900080E090E0A0E0B0E8282A392A4A2A5B2ABE
:100CA0009694879477946794C3CF81E090E0A0E016
:100CB000B0E0682A792A8A2A9B2AB6CF67FC05C049
:100CC000211431044104510449F280E490E0A0E091
:100CD000B0E0680E791E8A1E9B1EC0CFCB010E9419
:100CE0001D08DC01CB01BC01CD01E2E1A0960C9412
:100CF0000E0AA8E1B0E0EFE7F6E00C94FA09DC0197
:100D0000CB01898B9A8BAB8BBC8B2D8B3E8B4F8B06
:100D1000588FBE016F5F7F4FCE0141960E9405093B
:100D20008E01075F1F4FB801CE0145960E9405094D
:100D3000FE0131962981223008F45FC039853230B6
:100D400010F4B8017BC081819A8589278183243082
:100D500009F455C0223009F452C0343009F454C0AB
:100D6000323009F458C06B817C818B859C85681B6F
:100D7000790B2D813E814F815885ED84FE840F854E
:100D800018892E153F054007510730F4220F331FF5
:100D9000441F551F615070407C836B8380E090E05E
:100DA000A0E0B0E4AA24BB2465012E153F0540074E
:100DB000510740F0A82AB92ACA2ADB2A2E193F096E
:100DC000400B510BB695A79597958795220F331F2A
:100DD000441F551F0097A105B10539F7D601C5017C
:100DE0008F779070A070B07080349105A105B10527
:100DF000A9F0A482B582C682D782BF011FC0231783
:100E0000E1F760E071E01AC01D821E821F82188621
:100E10001C821B82F2CF84E08983EFCFA7FC05C040
:100E2000211531054105510521F380E490E0A0E052
:100E3000B0E0A80EB91ECA1EDB1EDBCFCB010E949C
:100E40001D08DC01CB01BC01CD01EAE068960C94E1
:100E5000160AA8E1B0E0EFE2F7E00C94000ADC012A
:100E6000CB01898B9A8BAB8BBC8B2D8B3E8B4F8BA5
:100E7000588FBE016F5F7F4FCE0141960E940509DA
:100E80008E01075F1F4FB801CE0145960E940509EC
:100E90008981823018F08985823018F42FEF3FEF76
:100EA00009C0B801CE0101960E947F09282F33277F
:100EB00027FD3095C901E4E068960C941C0AA8E16E
:100EC000B0E0E5E6F7E00C94000ADC01CB01898B89
:100ED0009A8BAB8BBC8B2D8B3E8B4F8B588FBE016F
:100EE0006F5F7F4FCE0141960E9405098E01075F1B
:100EF0001F4FB801CE0145960E94050989818230B5
:100F000018F08985823018F42FEF3FEF09C0B8013F
:100F1000CE0101960E947F09282F332727FD3095A7
:100F2000C901E4E068960C941C0AA8E1B0E0EBE982
:100F3000F7E00C94000ADC01CB01898B9A8BAB8B18
:100F4000BC8B2D8B3E8B4F8B588FBE016F5F7F4FBD
:100F5000CE0141960E9405098E01075F1F4FB8011F
:100F6000CE0145960E9405098981823018F0898555
:100F7000823018F421E030E009C0B801CE010196BA
:100F80000E947F09282F332727FD3095C901E4E00F
:100F900068960C941C0AACE0B0E0E1EDF7E00C942C
:100FA000020ADC01CB0189879A87AB87BC87BE0127
:100FB0006F5F7F4FCE0109960E94050989818230BB
:100FC00011F0823028F460E070E080E090E031C001
:100FD000843039F02B813C8137FDF5CF2F3131053D
:100FE0006CF08A81882329F060E070E080E090E86E
:100FF00020C06FEF7FEF8FEF9FE71BC08EE190E087
:10100000821B930B2D813E814F81588504C05695DC
:101010004795379527958A95D2F78A81882339F0A5
:1010200050954095309521953F4F4F4F5F4FCA01E6
:10103000B901E2E02C960C941E0AA0E0B0E0E3E2D5
:10104000F8E00C94F809882499245401DC01FC018F
:1010500024813581468157818181082F112760E0E5
:1010600070E08C91823020F46FEF70E04061A4C09A
:10107000843009F464C0823009F463C0211531055D
:101080004105510509F498C0FD0182819381FFEF6C
:1010900082389F070CF050C0A2E8EA2EAFEFFA2E7C
:1010A000E81AF90A8AE1E816F1040CF06BC06B014A
:1010B00081E090E0A0E0B0E00E2C04C0880F991F02
:1010C000AA1FBB1F0A94D2F70197A109B109822375
:1010D0009323A423B5230097A105B10519F0F1E0EE
:1010E000CF2ED12C04C05695479537952795EA9475
:1010F000D2F7C601AA2797FDA095BA2F282B392B26
:101100004A2B5B2BDA01C9018F779070A070B07009
:1011100080349105A105B105D1F1215C3F4F4F4FBE
:101120005F4F2030E0E03E07E0E04E07E0E45E077E
:1011300008F161E070E01EC0803891053CF06FEF6F
:1011400070E020E030E040E050E036C0BC01615883
:101150007F4FDA01C9018F779070A070B070803432
:101160009105A105B105D1F0215C3F4F4F4F5F4F75
:1011700057FD1BC097E056954795379527959A954B
:10118000D1F71AC020E030E040E050E0BBCF27FFAD
:10119000C8CF205C3F4F4F4F5F4FC3CF27FFE8CFF3
:1011A000205C3F4F4F4F5F4FE3CF569547953795A4
:1011B00027956F5F7F4FDECF822E932E942F9F77E0
:1011C0008A2D8078A82EA92A962F979599279795EA
:1011D0008A2D8F77A82EA92A76956795962F9F77C7
:1011E0008B2D8078B82EB92A902F979599279795AF
:1011F0008B2D8F77B82EB92AD501C401BC01CD0142
:10120000ECE0CDB7DEB70C94140ACF93DF93FC016A
:10121000DB01408151812281622F6F7770E0221FB4
:101220002227221F9381892F880F822B282F332773
:10123000991F9927991FED0199832115310541F4D3
:101240004115510561057105E1F482E08C9354C0AC
:101250002F3F310509F441C02F573040FD01338342
:10126000228383E08C9387E0440F551F661F771F0E
:101270008A95D1F77064ED014C835D836E837F8323
:101280003BC022E83FEFF901C7E0440F551F661F3E
:10129000771FCA95D1F783E08C93403080E05807E0
:1012A00080E0680780E4780778F4440F551F661FD4
:1012B000771F21503040F9014030C0E05C07C0E0AA
:1012C0006C07C0E47C0788F3ED01FB83EA83FD0132
:1012D00044835583668377830FC0411551056105AB
:1012E000710519F484E08C9307C064FF03C081E0AA
:1012F0008C93C1CF1C92BFCFDF91CF9108950F93F4
:101300001F93CF93DF93FC01DB018081823018F0C3
:101310009C91923018F461E070E05EC08430C1F0BE
:10132000843001F1943009F447C0823009F44BC095
:10133000823009F44EC09230A9F04181ED018981DB
:101340004817B9F0442389F08FEF9FEFBC0144C0E8
:10135000943031F7EB018981682F77278181681BF1
:1013600071093AC08181882379F781E090E0BC015E
:1013700033C022813381ED018A819B8182179307DB
:101380000CF3281739079CF00481158126813781D9
:10139000FD016481758186819781601771078207DD
:1013A000930780F2061717072807390778F44423B4
:1013B00059F281E090E0DBCFFD018181882321F2A9
:1013C00081E090E0D4CF923009F0B2CF60E070E0DD
:1013D00003C0ED018981F2CFCB01DF91CF911F9145
:1013E0000F9108952F923F924F925F926F927F924A
:1013F0008F929F92AF92BF92CF92DF92EF92FF9225
:101400000F931F93CF93DF93CDB7DEB7CA1BDB0BD0
:101410000FB6F894DEBF0FBECDBF09942A88398875
:1014200048885F846E847D848C849B84AA84B9847C
:10143000C884DF80EE80FD800C811B81AA81B98188
:10144000CE0FD11D0FB6F894DEBF0FBECDBFED019C
:041450000895FFCF2D
:08145400000000000000000090
:00000001FF
